:100000000C948B000C94B3000C94B3000C94B300CC
:100010000C94B3000C94B3000C94B3000C94B30094
:100020000C94B3000C94B3000C94B3000C94B30084
:100030000C94B3000C94620E0C94B3000C94B300B7
:100040000C94B3000C94B3000C949B1B0C94B30061
:100050000C94B3000C94B3000C94B3000C94B30054
:100060000C94B3000C94B3000C94B3000C94B30044
:100070000C94B3000C94B3000C94B3000000000087
:10008000240027002A0000000000250028002B0083
:1000900000000000230026002900040404040404D6
:1000A0000404020202020202030303030303010227
:1000B00004081020408001020408102001020408F6
:1000C00010200000000700020100000304060000E9
:1000D000000000000000494E46494E4954594E4127
:1000E0004ECDCCCC3D0AD7233C17B7D13877CC2B9B
:1000F000329595E6241FB14F0A000020410000C848
:100100004200401C4620BCBE4CCA1B0E5AAEC59DC8
:100110007400FA09EC1E11241FBECFEFD0E1DEBF40
:10012000CDBF11E0A0E0B1E0E6EEF4E402C005903E
:100130000D92A233B107D9F715E0A2E3B1E001C0F7
:100140001D92A53BB107E1F711E0C6E1D1E004C083
:100150002297FE010E942B22C231D107C9F70E94CB
:100160009D1D0C9471220C940000A0E0B0E0EBEB1C
:10017000F0E00C944022EC015B016115710519F06F
:10018000FB0191838083F9908F2D90E00E942F22B4
:10019000892BC9F7FDE2FF1621F4F990EE24E394D0
:1001A00005C02BE2F21609F4F990EE248E010150FD
:1001B0001040C80166ED70E043E050E00E94440347
:1001C000892B01F58E010E5F1F4FC80169ED70E0AC
:1001D00045E050E00E944403892B19F48E01095F29
:1001E0001F4FA114B10419F0F50111830083E0FC45
:1001F00004C070E090E080E814C070E090E080E817
:100200006FEF08C1C8016EED70E043E050E00E945E
:100210004403892B69F4A114B10429F470E090E03F
:1002200080EC6FE7F7C02296F501D183C083F6CF4B
:100230008824992440E050E060E070E0EF2DE05326
:10024000EA30A0F5F2E0EF2A8E2D90E09C012870B4
:100250003070E2FE06C0232B79F50894811C911CB6
:100260002BC0232B19F0089481089108DB01CA01E7
:1002700012E0880F991FAA1FBB1F1A95D1F7480FCC
:10028000591F6A1F7B1F440F551F661F771F4E0F94
:10029000511D611D711D483929E9520729E962077D
:1002A00029E1720748F084E0E82A06C0EE3F31F405
:1002B000E3FC39C098E0E92AF990C0CFE53311F0AA
:1002C000E53189F529912D3219F4E0E1EE2A05C0D6
:1002D0002B3219F081E090E003C0299182E090E098
:1002E000E22FE053EA3018F0C81BD90B1CC020E005
:1002F00030E0FCE020383F075CF4C901880F991F0B
:10030000880F991F280F391F220F331F2E0F311D01
:10031000E991E053EA3068F3E4FE03C0309521959B
:100320003F4F820E931ECE2CDD24E1FE07C0A114A8
:10033000B10421F02197F501D183C083CB01BA012B
:100340000E9428207B018C01F3E0CF22DD2423E0F2
:10035000C216D10421F417FB109517F91095570117
:100360006801C801B70120E030E040E050E00E94A1
:100370008B1F882309F44AC097FE0DC025EFE22E9B
:1003800020E0F22E9094819491089394C0E2D0E002
:1003900000E010E012C09DE0E92E91E0F92EF6CFCA
:1003A000F7012591359145915491C601B5010E94FF
:1003B000DE205B016C018C1A9D0A8C169D0684F769
:1003C000D595C7950F5F1F4F0630110529F08CEFAB
:1003D0009FEFE80EF91EF1CFC501D6017C018D011A
:1003E0008C2D880F8D2D881F8F3F51F0C601B501D0
:1003F00020E030E040E050E00E948B1F882331F481
:1004000082E290E09093B4058093B3057E2D9F2DFA
:10041000802F612F272F392F482F562FB901CA015E
:10042000CDB7DEB7ECE00C945C222F923F925F9246
:100430006F927F928F929F92AF92BF92CF92DF92F4
:10044000EF92FF920F931F93CF93DF938C011B01C9
:10045000EA016115710519F0FB01918380832097F2
:1004600049F0CE010297839728F020E030E040E089
:1004700050E0F6C0F801A1908F018A2D90E00E9413
:100480002F22892BB9F7FDE2AF1631F4F801A190C4
:100490008F015524539407C0FBE2AF1619F4F801FD
:1004A000A1908F015524209719F0C031D105C1F4D6
:1004B000F0E3AF1679F4F8018081883711F08835C0
:1004C00049F4F801A1800E5F1F4FF2E05F2AC0E1FE
:1004D000D0E006C0209721F480E3A816E9F427C0F5
:1004E000C830D10531F1C930D10524F4C230D1056D
:1004F00031F50CC0CA30D10589F0C031D105F9F40D
:10050000C12CD12CE12CB8E0FB2E28C0C12CD12C61
:10051000E12CA0E4FA2E22C0CAE0D0E0FCECCF2E01
:10052000FCECDF2EFCECEF2EFCE0FF2E17C0C8E049
:10053000D0E0C12CD12CE12CE0E1FE2E0FC09E01B9
:10054000442737FD4095542F60E070E080E090E84C
:100550000E94D821C901DA016C017D0120E030E060
:1005600040E050E060E03E01882477FC8094982CC5
:1005700070EDB72EBA0CE9E0EB1570F48A2D8154BA
:100580008A3118F499ECB92E06C08A2D81568A3129
:1005900050F589EAB82EBA0C8B2D90E08C179D0788
:1005A00014F56F3FE1F0C216D306E406F506B0F08D
:1005B000CA01B901A40193010E94A6219B01AC01CB
:1005C0002B0D311D411D511D2130F0E03F07F0E0A2
:1005D0004F07F0E85F0710F461E001C06FEFF8012A
:1005E000A1908F01C5CF2114310481F0662331F031
:1005F00001501040F1011183008308C051FE1AC060
:1006000002501040F1011183008314C067FF12C033
:1006100050FC05C02FEF3FEF4FEF5FE704C020E035
:1006200030E040E050E882E290E09093B40580939F
:10063000B30516C050FE08C05095409530952195E1
:100640003F4F4F4F5F4F0CC057FF0AC082E290E010
:100650009093B4058093B3052FEF3FEF4FEF5FE723
:10066000B901CA01DF91CF911F910F91FF90EF90D7
:10067000DF90CF90BF90AF909F908F907F906F90C2
:100680005F903F902F900895FB01DC014150504056
:1006900088F08D9181341CF08B350CF4805E65916F
:1006A00061341CF06B350CF4605E861B611171F3D4
:1006B000990B0895881BFCCF2F923F924F925F9227
:1006C0006F927F928F929F92AF92BF92CF92DF9262
:1006D000EF92FF920F931F93DF93CF93CDB7DEB7C7
:1006E0002E970FB6F894DEBF0FBECDBF9E878D87C5
:1006F0008B017A01FB016081718182819381FA0112
:1007000020813181428153810E94DE205B016C0196
:10071000F8016481758186819781F7012481358193
:10072000468157810E94DE203B014C01F801608523
:10073000718582859385F7012085318542855385B2
:100740000E94DE201B012C01F801648575858685D9
:100750009785F70124853585468557850E94DE20DB
:1007600069877A878B879C87F8016089718982897C
:100770009389F70120893189428953890E94DE20BB
:100780007B018C01C601B50120E030E040E050E083
:100790000E94DA2088234CF0C601B50120E030E049
:1007A00040E05FE30E94271F08C0C601B50120E0BA
:1007B00030E040E05FE30E94261F0E94F71F69833C
:1007C0007A838B839C83C401B30120E030E040E056
:1007D00050E00E94DA2088234CF0C401B30120E0ED
:1007E00030E040E05FE30E94271F08C0C401B3016E
:1007F00020E030E040E05FE30E94261F0E94F71FE8
:100800006D837E838F839887C201B10120E030E041
:1008100040E050E00E94DA2088234CF0C201B10190
:1008200020E030E040E05FE30E94271F08C0C201E3
:10083000B10120E030E040E05FE30E94261F0E940B
:10084000F71F3B014C0169857A858B859C8520E0EB
:1008500030E040E050E00E94DA2088235CF06985B7
:100860007A858B859C8520E030E040E05FE30E9444
:10087000271F0AC069857A858B859C8520E030E03A
:1008800040E05FE30E94261F0E94F71F5B016C019E
:10089000C801B70120E030E040E050E00E94DA20DB
:1008A00088234CF0C801B70120E030E040E05FE36E
:1008B0000E94271F08C0C801B70120E030E040E0D7
:1008C0005FE30E94261F0E94F71F29813A814B8116
:1008D0005C81ED85FE8520833183428353832D81A6
:1008E0003E814F81588524833583468357836086B4
:1008F000718682869386A486B586C686D786608BE7
:10090000718B828B938BCF012E960FB6F894DEBF3E
:100910000FBECDBFCF91DF911F910F91FF90EF9050
:10092000DF90CF90BF90AF909F908F907F906F900F
:100930005F904F903F902F900895882321F48091ED
:1009400081008B7F29C0813049F4809181008B7FA9
:100950008093810080918100826015C0823049F4CB
:10096000809181008B7F80938100809181008260E3
:1009700018C0833071F4809181008460809381007D
:10098000809181008D7F80938100809181008E7F96
:100990000DC08091810084608093810080918100EE
:1009A0008D7F8093810080918100816080938100A0
:1009B0000895E0E8F0E01082A1E8B0E01C92109207
:1009C000820010926F008C918F7E8C938C91886046
:1009D0008C9380818D7F808380818E7F80838081D6
:1009E0008F77808380818F7B808380818F7D8083E0
:1009F00080818F7E808384E00E949D048FEF9FEF33
:100A000090938900809388000895FC0180819181F2
:100A1000A281B381803020E0920721E0A20720E08C
:100A2000B2070CF441C0893F2FEF920727E0A207DD
:100A300020E0B20744F453E0B595A79597958795C4
:100A40005A95D1F731C0813C2FEF92072FE3A207CF
:100A500020E0B20744F446E0B595A79597958795B1
:100A60004A95D1F721C081302FEF92072FEFA207CF
:100A700020E0B2073CF4892F9A2FAB2FBB27A7FDAC
:100A8000BA9512C081302CEF92072FEFA20723E016
:100A9000B2071CF0EFEFFFEF08C02AE0B595A7956D
:100AA000979587952A95D1F7FC01CF010895EF928C
:100AB000FF920F931F93DF93CF9300D000D0CDB759
:100AC000DEB77B018C0164E0EE0CFF1C001F111FE0
:100AD0006A95D1F7E982FA820B831C83CE010196D5
:100AE0000E940505909389008093880080E0E816B5
:100AF00080E0F80681E0080780E0180714F480E041
:100B000022C089EFE8168FEFF80687E0080780E03B
:100B1000180714F481E017C081ECE8168FEFF8068F
:100B20008FE3080780E0180714F482E00CC081E02E
:100B3000E8168FEFF8068FEF080780E0180714F02B
:100B400084E001C083E00E949D040F900F900F90FD
:100B50000F90CF91DF911F910F91FF90EF9008952B
:100B6000AF92BF92CF92DF92EF92FF920F931F93BB
:100B7000DF93CF9300D0CDB7DEB78C017B016A0144
:100B80005901BE016F5F7F4F4AE050E00E9415029D
:100B900029813A81201B310B121613065CF4F701F0
:100BA00071836083F601808191818A299B299183D9
:100BB000808303C0F70111821082C9010F900F904A
:100BC000CF91DF911F910F91FF90EF90DF90CF9029
:100BD000BF90AF900895AF92BF92CF92DF92EF9205
:100BE000FF920F931F93DF93CF9300D0CDB7DEB763
:100BF0008C017B016A015901BE016F5F7F4F0E942A
:100C0000B50029813A81201B310B121613066CF4B2
:100C1000F7016083718382839383F60180819181E0
:100C20008A299B299183808309C080E090E0A0E01D
:100C3000B0E0F70180839183A283B383C9010F9051
:100C40000F90CF91DF911F910F91FF90EF90DF9068
:100C5000CF90BF90AF9008952F923F924F925F92A6
:100C60006F927F928F929F92AF92BF92CF92DF92BC
:100C7000EF92FF920F931F93DF93CF93CDB7DEB721
:100C800064970FB6F894DEBF0FBECDBF8B015A8BB1
:100C9000498BFC01119211926F017C019C012C5F28
:100CA0003F4F388B2F87FC013696FE87ED879C01DE
:100CB000285D3F4F3C872B87FC013896FA87E987F0
:100CC0009C01245F3F4F38872F83FC017096FE8381
:100CD000ED839C012C5E3F4F3C832B83FC017C9673
:100CE000FA83E983B0E22B2E312C280E391EA4E2C0
:100CF0004A2E512C480E591EFCE26F2E712C680EA4
:100D0000791EE0E38E2E912C880E991E78E1A72E95
:100D1000B12CA80EB91E1C8A1B8ACCC0EB89FC8999
:100D2000E00FF11FE081E03509F456C0E13594F49D
:100D3000E73441F1E83434F4E53409F4A9C0E63489
:100D4000F1F48BC0EA3409F47EC0ED3429F1E934C2
:100D5000B1F46EC0E43569F1E5354CF4E23509F4DF
:100D600086C08B899C890196E33574F58AC0E93584
:100D700009F448C0EA3509F450C0E835C1F180E013
:100D800090E091C08B899C890196800F911FB601DC
:100D9000A70121E030E00AC08B899C890196800F71
:100DA000911F6F857889A70122E030E00E94B0058D
:100DB0007AC08B899C890196800F911F6D857E85F5
:100DC000A70120E030E4F2CF800F911F6B857C8576
:100DD000A70120E034E065C08B899C890196800FD3
:100DE000911F69857A85A70124E030E05AC08B897C
:100DF0009C890196800F911F6F817885A70128E05B
:100E000030E04FC08B899C890196800F911F6D81C6
:100E10007E81A70120E130E044C08B899C89019646
:100E2000800F911F6B817C81A70120E230E039C0E7
:100E30008B899C890196800F911F69817A81A70116
:100E400020E430E02EC08B899C890196800F911F91
:100E5000B101A70120E830E024C08B899C8901966C
:100E6000800F911FB201A70120E032E01AC08B89E8
:100E70009C890196800F911FB301A70120E030E10A
:100E800010C0800F911FB401A70120E038E009C015
:100E90008B899C890196800F911FB501A70120E0E5
:100EA00030E20E94EB0501962B893C89280F391FFF
:100EB0003C8B2B8B8B899C89E989FA898E179F073C
:100EC0000CF42CCF64960FB6F894DEBF0FBECDBFE6
:100ED000CF91DF911F910F91FF90EF90DF90CF9016
:100EE000BF90AF909F908F907F906F905F904F904A
:100EF0003F902F900895EF92FF920F931F937C01E4
:100F0000FC0185890E94241B8C01F70185890E94C0
:100F1000241B080F191FF70185890E94241B800FCD
:100F2000911F63E070E00E94C521CB011F910F91DA
:100F3000FF90EF9008950E947B07AA2797FDA09548
:100F4000BA2FBC01CD010E942A2020E030E040EA07
:100F500050E40E94DE2020E030E048EC52E40E94A1
:100F6000DE2020E030E040E85AE30E94DE200E94CC
:100F7000F71FCB010895CF93DF93EC010E949B07ED
:100F80009C0189819A812817390714F46E8108C061
:100F90008B819C812817390714F060E001C06D81B6
:100FA0008F81861729F06F838B8970E00E94421B26
:100FB000DF91CF91089580913201909133010E9489
:100FC000BB0780913401909135010E94BB070895C1
:100FD000CF93DF93EC011A860E949B079C878B8737
:100FE0001DC00E94DB078A858F5F8A87853180F06C
:100FF000CE010E949B079C019E878D878B859C85D7
:101000008217930714F081E014C03C872B871A865F
:1010100068EE73E080E090E00E94E31BCE010E9446
:101020009B0729813A812550304082179307CCF2E3
:1010300080E0DF91CF910895FF920F931F93CF939C
:10104000DF93EC01F62E8A010E94E807882381F0E5
:1010500080EA95E060E071E00E94881CCE010E9469
:101060009B07BC0180EA95E04AE050E00E94821DA7
:10107000F88A8E896F2D0E94881A8F8961E00E94FC
:10108000881AB801882777FD8095982F0E94E31B66
:101090008F8960E00E94881ADF91CF911F910F9194
:1010A000FF90089583E161E00E94881A83E161E086
:1010B0000E94881A8FE161E00E94881A0895CF93F8
:1010C000DF93EC01C859DF4F88819981AA81BB81E8
:1010D000C856D0400097A105B10521F083E160E03A
:1010E0000E94881AC459DF4F88819981AA81BB81E7
:1010F000CC56D0400097A105B10521F083E160E016
:101100000E94881AC059DF4F88819981AA81BB81CA
:10111000C057D0400097A105B10521F08FE160E0F4
:101120000E94881ACC58DF4F88819981AA81BB819F
:101130000097A105B10571F0E0913601F0E0EE0FE6
:10114000FF1FEE5CFE4F0190F081E02D808D60E08E
:101150000E94881ADF91CF910895CF93DF93EC011D
:10116000CA55DF4F8881C65AD0408823E1F5CC5656
:10117000DF4F82E169910E94881A86E169910E949D
:10118000881A8EE169910E94881A8881C759D040D7
:10119000E0913601882369F0F0E0EE0FFF1FEE5C6E
:1011A000FE4F0190F081E02D81E08787818961E029
:1011B0000BC0F0E0EE0FFF1FEE5CFE4F0190F081E0
:1011C000E02D1786818960E00E94881ACE010E9476
:1011D0005F0868EE73E080E090E00E945705C85514
:1011E000DF4F81E08883DF91CF9108956F927F92E6
:1011F0008F92AF92CF92EF920F93DF93CF93CDB7B1
:10120000DEB73C01862FF301618B428B238B048B6D
:10121000E58AC68AA78A808E61E00E94681AF30177
:10122000828961E00E94681AF301838961E00E946B
:10123000681AF301858960E00E94681AF3018689C3
:1012400061E00E94681AF301878961E00E94681AD0
:10125000F301818961E00E94881AF301838960E0CB
:1012600070E00E94421BF301828960E070E00E94FE
:10127000421BF301868960E00E94881AF301878986
:1012800060E00E94881AF301808D61E00E94681A74
:10129000F301808D61E00E94881AF301108280E4DE
:1012A00085838FEF86831782108A81E08787128279
:1012B000118280E090E06AE070E00E94C5217483B2
:1012C0006383CF91DF910F91EF90CF90AF908F908C
:1012D0007F906F9008950F931F938C0108551F4FB7
:1012E000F801108202501040F801108202511040A3
:1012F00081E0F80181938193819381938F018083B1
:101300000859104080E090E0A0E0B0E0F801848B44
:10131000958BA68BB78B808F918FA28FB38F848F85
:10132000958FA68FB78F80A391A3A2A3B3A380E0CC
:1013300090E0AAE7B4E484A395A3A6A3B7A38FE0A3
:1013400061E00E94681A82E161E00E94681A87E108
:1013500061E00E94681A86E161E00E94681A8DE1EE
:1013600061E00E94681A8EE161E00E94681A83E1E0
:1013700061E00E94681A83E161E00E94681A8FE1CF
:1013800061E00E94681AC8010E94520884E160E08E
:101390000E94681A89E160E00E94681A81E060E0BA
:1013A0000E94681A8BE49AEEAFEFB0E4F8018083F4
:1013B0009183A283B38384839583A683B78380E0DC
:1013C00090E0A0EAB3E480879187A287B3878AE69A
:1013D0009CEBA4E3BFE384879587A687B78780E06B
:1013E00090E0A0E8BFE3808B918BA28BB38B1F9121
:1013F0000F9108958F92AF92CF92EF920F938DE35A
:1014000092E060E044E028E107E0B3E0EB2EA6E0E4
:10141000CA2EF5E0AF2E88248A940E94F60886E54D
:1014200092E060E14CE02EE003E0E4E0EE2E71E1BA
:10143000C72E5DE0A52E33E0832E0E94F6088FE6CE
:1014400092E00E946B0988E193E00E946B0981ECB5
:1014500093E00E946B098AE694E00E946B090F9169
:10146000EF90CF90AF908F900895AF92BF92CF92B0
:10147000DF92EF92FF920F931F93B62EC016D10604
:10148000E206F30611F480E00DC0862F0E94D51A03
:10149000892B39F08B2D0E94D51A892B11F08A2DBA
:1014A000A11081E01F910F91FF90EF90DF90CF90FE
:1014B000BF90AF9008952F923F924F925F926F929C
:1014C0007F928F929F92AF92BF92CF92DF92EF92D4
:1014D000FF920F931F93DF93CF93CDB7DEB7AC97F7
:1014E0000FB6F894DEBF0FBECDBF88559F4FDC010D
:1014F0008C91A85AB040BCA7ABA7882309F4C9C3F4
:10150000A05CBF4FBA83A983EBA5FCA5EC5AFF4FA3
:10151000FC83EB832BA53CA52C563F4F3E832D83AC
:101520008BA59CA587569F4F98878F83ABA5BCA59D
:10153000AC5BBF4FBA87A987EBA5FCA5E85AFF4F64
:10154000FC87EB872BA53CA52B563F4F3E872D876D
:101550008BA59CA586569F4F988B8F87ABA5BCA566
:10156000A85BBF4FBA8BA98BEBA5FCA5E45AFF4F34
:10157000FC8BEB8B2BA53CA52A563F4F3E8B2D8B2E
:101580008BA59CA585569F4F988F8F8B3CE4232E6F
:10159000312CABA5BCA52A0E3B1EA05ABF4FBA8F5B
:1015A000A98FEBA5FCA5E956FF4FFC8FEB8F2BA570
:1015B0003CA524563F4F3E8F2D8F20E5622E712C87
:1015C0008BA59CA5680E791E8C599F4F98A38F8F71
:1015D000ABA5BCA5A856BF4FBAA3A9A3EBA5FCA574
:1015E000E356FF4FFCA3EBA397EA892E912C2BA582
:1015F0003CA5820E931E28593F4F3EA32DA38BA5D9
:101600009CA584589F4F98A78FA38EE9482E512CF4
:10161000ABA5BCA54A0E5B1EA459BF4FBAA7A9A78C
:10162000E981FA810081118122813381AB81BC8102
:10163000CD90DD90ED90FC908BA59CA564E145E1FB
:10164000ED81FE81A0800E94350AAF81B8858C9320
:10165000E985FA850081118122813381AB85BC85C2
:10166000CD90DD90ED90FC908BA59CA569E14AE1C1
:10167000ED85FE85A0800E94350AAF85B8898C93E0
:10168000E989FA890081118122813381AB89BC8982
:10169000CD90DD90ED90FC908BA59CA561E042E0A3
:1016A000ED89FE89A0800E94350AAF89B88D8C93A0
:1016B000F1010081118122813381A98DBA8DCD90F4
:1016C000DD90ED90FC908BA59CA56FEF4FEFEB8D1F
:1016D000FC8DA0800E94350AAD8DBE8D8C93F301E8
:1016E0000081118122813381AF8DB8A1CD90DD9031
:1016F000ED90FC908BA59CA56FEF4FEFE9A1FAA1AF
:10170000A0800E94350AABA1BCA18C93F401108289
:10171000AF81B8858C91882309F45CC0EDA1FEA14E
:1017200080819181A281B381EFA1F8A520813181CF
:1017300042815381820F931FA41FB51F8083918321
:10174000A283B383181619061A061B060CF042C0B2
:101750008FE061E00E94881A85E090E00E940D1CF5
:101760008FE060E00E94881A81E0D4018C93EFA1A1
:10177000F8A580819181A281B381F201208131811C
:1017800042815381821B930BA40BB50BEFA1F8A5EB
:1017900080839183A283B383AD81BE818C91E981E3
:1017A000FA812081318142815381882349F02F5F62
:1017B0003F4F4F4F5F4F20833183428353830AC093
:1017C0002150304040405040E981FA8120833183EC
:1017D00042835383AF85B8898C91882309F45AC01A
:1017E0000BA51CA500581F4FE9A5FAA58081918182
:1017F000A281B381F8012081318142815381820F1E
:10180000931FA41FB51F80839183A283B3831816EF
:1018100019061A061B06F4F587E161E00E94881A92
:1018200085E090E00E940D1C87E160E00E94881A2C
:1018300081E0D4018C93F80180819181A281B381F0
:10184000F2012081318142815381821B930BA40BD1
:10185000B50BF80180839183A283B383AD85BE85E8
:101860008C91882351F0E985FA8580819181A2814C
:10187000B3810196A11DB11D09C0E985FA8580815A
:101880009181A281B3810197A109B10980839183DC
:10189000A283B383AF89B88D8C91882309F460C08B
:1018A0000BA51CA50C571F4FEBA5FCA5E059FF4F3E
:1018B00080819181A281B381E057F040FCA7EBA722
:1018C000F8012081318142815381820F931FA41F2F
:1018D000B51F80839183A283B383181619061A0655
:1018E0001B06F4F58DE161E00E94881A85E090E026
:1018F0000E940D1C8DE160E00E94881A81E0D401F5
:101900008C93F80180819181A281B381F2012081C1
:10191000318142815381821B930BA40BB50BF801DB
:1019200080839183A283B383AD89BE898C91882300
:1019300051F0E989FA8980819181A281B381019670
:10194000A11DB11D09C0E989FA8980819181A28117
:10195000B3810197A109B10980839183A283B383E5
:10196000AD8DBE8D8C91882309F46CC008E8E02E03
:10197000F12CEBA5FCA5EE0EFF1EEC58FF4F80816D
:101980009181A281B381E457F040FCA7EBA7F70156
:101990002081318142815381820F931FA41FB51F83
:1019A00080839183A283B383181619061A061B0637
:1019B0000CF048C0E0913601F0E0EE0FFF1FEE5C46
:1019C000FE4F00811181D80152968C9161E00E94F6
:1019D000881A85E090E00E940D1CF801828960E081
:1019E0000E94881A81E0D4018C93F7018081918153
:1019F000A281B381F2012081318142815381821B16
:101A0000930BA40BB50BF70180839183A283B3835F
:101A1000AB8DBC8D8C91882349F0F101808191813F
:101A2000A281B3810196A11DB11D08C0F101808181
:101A30009181A281B3810197A109B109808391832A
:101A4000A283B383ABA1BCA18C91882309F44AC0C3
:101A5000EBA5FCA5E457FF4F2BA53CA528583F4F0D
:101A6000D9012D913D914D915C911397A857B040AC
:101A7000BCA7ABA780819181A281B381280F391FB8
:101A80004A1F5B1F20833183428353831216130640
:101A9000140615063CF5D201ED90FD900D911C91B8
:101AA0002E193F09400B510B20833183428353830E
:101AB000E9A1FAA18081882349F0F3018081918115
:101AC000A281B3810196A11DB11D08C0F3018081DF
:101AD0009181A281B3810197A109B109808391838A
:101AE000A283B383D4018C91882309F487C0EBA52A
:101AF000FCA5E057FF4F2081318142815381E0599D
:101B0000F040FCA7EBA78F010E551F4F2230310587
:101B1000410551056CF0D3016D917D918D919C91A2
:101B20000E94A621F80160837183828393830AC097
:101B3000F30180819181A281B381F8018083918337
:101B4000A283B383ABA5BCA5DC966D917D918D91ED
:101B50009C91DF9720EC31EE44E65CE40E94DE20AD
:101B60005B016C01EBA5FCA5EE55FF4F6081718117
:101B7000828193810E942A207B018C01F201608185
:101B80007181828193810E942A209B01AC01C8014E
:101B9000B7010E94DE209B01AC01C601B5010E9485
:101BA0008F1F7B018C0120E030E040E050E00E947C
:101BB000DA2088234CF0C801B70120E030E040E093
:101BC0005FE30E94271F08C0C801B70120E030E092
:101BD00040E05FE30E94261F0E94F71F2BA53CA553
:101BE0002E553F4FD9016D937D938D939C93139701
:101BF000A25AB040BCA7ABA70E945705F401808150
:101C0000882331F4ABA1BCA18C91882309F008CDC5
:101C1000EBA5FCA5E756FF4F8081E959F040FCA7F2
:101C2000EBA7882319F5E656FF4F8081EA59F0406B
:101C3000FCA7EBA78823D1F4E556FF4F8081EB5931
:101C4000F040FCA7EBA7882389F4E456FF4F80817E
:101C5000EC59F040FCA7EBA7882341F4E356FF4F73
:101C60008081ED59F040FCA7EBA701C081E0EBA516
:101C7000FCA5E855FF4F80838081882351F48BA514
:101C80009CA50E94520868EE73E080E090E00E94FC
:101C90005705AC960FB6F894DEBF0FBECDBFCF91FF
:101CA000DF911F910F91FF90EF90DF90CF90BF9049
:101CB000AF909F908F907F906F905F904F903F90EC
:101CC0002F9008951F920F920FB60F9211241F9319
:101CD0002F933F934F935F936F937F938F939F9334
:101CE000AF93BF93EF93FF9380916F008D7F8093AD
:101CF0006F00E0914A01F0E0EE0FFF1FEF5BFE4F37
:101D00000190F081E02DE855FF4F8081882361F03C
:101D1000E0914A01F0E0EE0FFF1FEF5BFE4F808184
:101D200091810E945B0A22C090914A0180914901F1
:101D3000981799F5E0914A01F0E0EE0FFF1FEF5B75
:101D4000FE4F0190F081E02DE855FF4F8081882300
:101D500021F50CC0E12FF0E0EE0FFF1FEF5BFE4F0F
:101D6000808191810E94AD0810934A0180916F009B
:101D7000826080936F00FF91EF91BF91AF919F912F
:101D80008F917F916F915F914F913F912F911F9113
:101D90000F900FBE0F901F90189510914A011F5F72
:101DA0001430C0F210E0D6CF2F923F924F925F9244
:101DB0006F927F928F929F92AF92BF92CF92DF925B
:101DC000EF92FF920F931F93DF93CF93CDB7DEB7C0
:101DD000A4970FB6F894DEBF0FBECDBF2C01362EF0
:101DE000272EDC015496862F972F9C01F90184E160
:101DF00001900D928150E1F726EA30E0420E531E29
:101E0000D2011C92EAE5FFEF4E0E5F1ED2015496FE
:101E10006D917D918D919C91579720914B013091BF
:101E20004C0140914D0150914E010E94261F5B01D3
:101E30006C01E894D7F8F201608D718D828D938DDD
:101E400020914F0130915001409151015091520128
:101E50000E94261F7B018C01E89417F9D2015C9641
:101E60006D917D918D919C915F972091530130915F
:101E7000540140915501509156010E94261F3B018B
:101E80004C01E89497F8F20160A171A182A193A19D
:101E900020915701309158014091590150915A01B8
:101EA0000E94261F9B01AC015F772D8F3E8F4F8FC5
:101EB00058A3D20194966D917D918D919C919797A5
:101EC00020915B0130915C0140915D0150915E0178
:101ED0000E94261F9B01AC015F7729A33AA34BA365
:101EE0005CA3D201D8962D933D934D935C93DB97E1
:101EF0002D8D3E8D4F8D58A1D4962D933D934D93AE
:101F00005C93D797F20160AA71AA82AA93AA9C96C1
:101F1000ED92FD920D931C939F97A0A6B1A6C2A629
:101F2000D3A6C601B501A60195010E94DE205B0182
:101F30006C01C801B701A80197010E94DE209B0136
:101F4000AC01C601B5010E94271F7B018C01C401B1
:101F5000B301A40193010E94DE209B01AC01C801E2
:101F6000B7010E94271FD201DC966D937D938D935C
:101F70009C93DF9720E030E040E050E00E948B1F10
:101F800018166CF06D8D7E8D8F8D98A19B01AC0124
:101F90000E94DE20F20164AF75AF86AF97AFD20129
:101FA000DC966D917D918D919C91DF9720E030E0E2
:101FB00040E050E00E948B1F18166CF069A17AA1D6
:101FC0008BA19CA19B01AC010E94DE20F20164AFB9
:101FD00075AF86AF97AFD201DC966D917D918D91F3
:101FE0009C91DF970E944521F20164AF75AF86AFE7
:101FF00097AFF42CE52C8E010F5F1F4FC801B20183
:102000004BE451E00E945C03D201A05CBF4FF80199
:1020100084E101900D928150E1F724E130E0420E1D
:10202000531E8E010F5F1F4FC8016F2D7E2DA20121
:102030000E945C0340E450E0440E551ED2016CEA5D
:102040007FEF460E571EF80184E101900D928150FA
:10205000E1F7F201EC5AFF4F80E490E0480E591E80
:1020600020813181428153812D8B3E8B4F8B588F44
:10207000F20180819181A281B38120EC3FEF420E79
:10208000531E4D895E896F89788D481B590B6A0BE9
:102090007B0B4D8B5E8B6F8B788F77FF0BC07095B2
:1020A0006095509541955F4F6F4F7F4F4D8B5E8B85
:1020B0006F8B788FF201E85AFF4F64E470E0460EB0
:1020C000571EE080F18002811381F20180819181AD
:1020D000A281B3812CEB3FEF420E531EE81AF90A9E
:1020E0000A0B1B0B17FF08C010950095F094E094A5
:1020F000E11CF11C011D111DF201E45AFF4F48E4DF
:1021000050E0440E551E6081718182819381698FF8
:102110007A8F8B8F9C8FF20180819181A281B38114
:1021200028EB3FEF420E531E498D5A8D6B8D7C8DEF
:10213000481B590B6A0B7B0B498F5A8F6B8F7C8F17
:1021400077FF0BC070956095509541955F4F6F4F2D
:102150007F4F498F5A8F6B8F7C8FF201E05AFF4F70
:102160006CE470E0460E571E80809180A280B380A0
:10217000F20180819181A281B38124EB3FEF420E75
:10218000531E881A990AAA0ABB0AB7FE08C0B0945F
:10219000A09490948094811C911CA11CB11CB2014C
:1021A00068587F4FF201EC59FF4F40E550E0440E74
:1021B000551E2081318142815381F20180819181BC
:1021C000A281B381E0EBFFEF4E0E5F1E281B390B9F
:1021D0004A0B5B0B57FF07C05095409530952195F2
:1021E0003F4F4F4F5F4FDB012D933D934D935C93DA
:1021F0001397E4E7F0E04E0E5F1ED2018D929D92A0
:10220000AD92BC921397298D3A8D4B8D5C8D5E9368
:102210004E933E932E93FD0112930293F292E2921B
:10222000DF012D893E894F89588D5E934E933E93F1
:102230002E932D01E8E9FFEF4E0E5F1EDA01C90172
:102240002E153F054007510714F4D801C7012EE9A8
:1022500030E0420E531EF20180839183A283B38348
:1022600022ED3FEF420E531EF20120813181428167
:10227000538160E97FEF460E571E82179307A4072C
:10228000B50714F4DA01C901EEE9F0E04E0E5F1E65
:10229000F20180839183A283B38326ED3FEF420E48
:1022A000531EF20120813181428153816CE87FEF1E
:1022B000460E571E82179307A407B50714F4DA01D8
:1022C000C901EEE9F0E04E0E5F1EF20180839183BA
:1022D000A283B38322E63FEF420E531E0097A1056F
:1022E000B10599F446EA50E0440E551E81E0D20152
:1022F0008C93ABE4B1E0232D322DC901FC0184E1C4
:1023000001900D928150E1F7A1C1B20168587F4F51
:10231000F201EC59FF4F20E530E0420E531E2081C0
:10232000318142815381F20180819181A281B38107
:10233000E0EBFFEF4E0E5F1E281B390B4A0B5B0BC9
:1023400057FF07C050954095309521953F4F4F4F0F
:102350005F4FDB012D933D934D935C931397F0E911
:10236000CF2ED12CC40CD51C21E030E040E050E051
:10237000D6012D933D934D935C931397E8E7F0E0DE
:102380004E0E5F1ED201ED90FD900D911C91E8E87C
:10239000FFEF4E0E5F1EEEE96E2E712C640C751C65
:1023A000D3012D913D914D915C912E153F05400734
:1023B00051070CF075C0C801B7010E94FA2149010C
:1023C0005A01F60180829182A282B382F3E08F16D5
:1023D0009104A104B1040CF454C082010C591F4FA4
:1023E000D8016D917D918D919C91A50194010E94E0
:1023F000FA2169017A01F8012083318342835383F2
:102400008201005B1F4FD8016D917D918D919C9150
:10241000A50194010E94FA21C901DA01F801808323
:102420009183A283B383A7019601281B390B4A0B22
:102430005B0B57FF07C050954095309521953F4F56
:102440004F4F5F4F68E770E0460E571ED2012D9345
:102450003D934D935C931397E8E8FFEF4E0E5F1E9C
:10246000F201E256FF4F80819181A281B3818217F0
:102470009307A407B507A4F42083318342835383D1
:102480000FC021E030E040E050E0D6012D933D93B5
:102490004D935C931397F301E082F18202831383DF
:1024A00082010C561F4FFF24D20154966D917D91ED
:1024B0008D919C91579720914B0130914C01409107
:1024C0004D0150914E010E94DA20882314F0FF2420
:1024D000F394F801F08282010B561F4FFF24D201C2
:1024E00058966D917D918D919C915B9720914F01B4
:1024F0003091500140915101509152010E94DA20D7
:10250000882314F0FF24F394F801F08282010A5624
:102510001F4FFF24D2015C966D917D918D919C910E
:102520005F97209153013091540140915501509192
:1025300056010E94DA20882314F0FF24F394F80156
:10254000F082820109561F4FFF24D20190966D91AF
:102550007D918D919C9193972091570130915801D5
:102560004091590150915A010E94DA20882314F0B9
:10257000FF24F394F801F082820108561F4FFF24D4
:10258000D20194966D917D918D919C919797209118
:102590005B0130915C0140915D0150915E010E94B0
:1025A000DA20882314F0FF24F394F801F0822EE956
:1025B00030E0420E531ED2016D917D918D919C9120
:1025C000E2E6FFEF4E0E5F1E22E030E040E050E01A
:1025D0000E94FA2150954095309521953F4F4F4FDD
:1025E0005F4FD201A458BF4F2C9311963C93119783
:1025F00012964C93129713965C931397F201E0583E
:10260000FF4F208331834283538324E830E0420E1E
:10261000531E8D919D910D90BC91A02DF20181933F
:102620009193A193B19381939193A193B19380835B
:102630009183A283B383ABE4B1E0232D322DC90192
:10264000FC0184E101900D928150E1F7A4960FB650
:10265000F894DEBF0FBECDBFCF91DF911F910F91D8
:10266000FF90EF90DF90CF90BF90AF909F908F90B2
:102670007F906F905F904F903F902F9008951F93A1
:10268000CF93DF93EC0106C061E070E080E090E062
:102690000E94E31B80914A01882329F4809149011B
:1026A000833059F4F1CF2091490180914A0130E003
:1026B00090E001972817390739F3109149011F5FFE
:1026C000143008F010E0E12FF0E0EE0FFF1FEF5B99
:1026D000FE4F80819181BE010E94D40E109349016A
:1026E000DF91CF911F910895CF93DF93EC019B0170
:1026F000A5EFB1E0EBE4F1E084E101900D928150AF
:10270000E1F788819981AA81BB818093F50190933B
:10271000F601A093F701B093F801F901808191814E
:10272000A281B3818093050290930602A0930702D1
:10273000B093080285EF91E00E943F13DF91CF91A3
:102740000895CF93DF93EC019B01A5EFB1E0EBE49B
:10275000F1E084E101900D928150E1F78881998147
:10276000AA81BB818093F9019093FA01A093FB01A8
:10277000B093FC01F90180819181A281B3818093A2
:10278000050290930602A0930702B093080285EF1A
:1027900091E00E943F13DF91CF910895CF93DF9393
:1027A000EC019B01A5EFB1E0EBE4F1E084E10190E5
:1027B0000D928150E1F788819981AA81BB81809334
:1027C000FD019093FE01A093FF01B0930002F90177
:1027D00080819181A281B38180930502909306024A
:1027E000A0930702B093080285EF91E00E943F1387
:1027F000DF91CF9108954F925F926F927F928F9267
:102800009F92AF92BF92CF92DF92EF92FF920F937F
:102810001F93DF93CF93CDB7DEB7C056D0400FB62E
:10282000F894DEBF0FBECDBFFC01AB0180818F32BB
:1028300009F448C580E090E0A0E0B0E08093E101B9
:102840009093E201A093E301B093E4018093E5014A
:102850009093E601A093E701B093E8018093E9012A
:102860009093EA01A093EB01B093EC018093ED010A
:102870009093EE01A093EF01B093F0018093F101EA
:102880009093F201A093F301B093F40189E092E0F8
:10289000BF010E942C062091090230910A02C90151
:1028A00083709074892B91F42115310579F0809112
:1028B00023019091240197FD09C090930C0280930D
:1028C0000B02216030930A02209309020091090251
:1028D00010910A0200FFECC380910B0290910C0250
:1028E0009093240180932301A1EEB1E0EBE4F1E0A9
:1028F00084E101900D928150E1F7809125019801CA
:1029000028703070882309F449C0232B81F080910E
:10291000150290911602A0911702B09118028093AF
:10292000E1019093E201A093E301B093E40104FF7D
:1029300010C08091190290911A02A0911B02B091CF
:102940001C028093E5019093E601A093E701B09308
:10295000E80105FF10C080911D0290911E02A09118
:102960001F02B09120028093E9019093EA01A093A5
:10297000EB01B093EC0115FF81C080912102909191
:102980002202A0912302B09124028093ED01909342
:10299000EE01A093EF01B093F00170C0232BD1F0B2
:1029A0006091E1017091E2018091E3019091E40175
:1029B0002091150230911602409117025091180291
:1029C0000E94271F6093E1017093E2018093E3016D
:1029D0009093E40104FF1AC06091E5017091E60153
:1029E0008091E7019091E8012091190230911A023B
:1029F00040911B0250911C020E94271F6093E50129
:102A00007093E6018093E7019093E80105FF1AC0F7
:102A10006091E9017091EA018091EB019091EC01E4
:102A200020911D0230911E0240911F025091200200
:102A30000E94271F6093E9017093EA018093EB01E4
:102A40009093EC0115FF1AC06091ED017091EE01B9
:102A50008091EF019091F0012091210230912202AA
:102A600040912302509124020E94271F6093ED01A0
:102A70007093EE018093EF019093F00111FF10C06D
:102A800080912D0290912E02A0912F02B0913002E0
:102A90008093F1019093F201A093F301B093F401BC
:102AA00080910B0290910C028130910539F18C31AB
:102AB000910549F1892B09F01BC2E090F101F090DA
:102AC000F2010091F3011091F40180E090E8ABE392
:102AD000B5E48093F1019093F201A093F301B093D8
:102AE000F40181EE91E00E943F13E092F101F09237
:102AF000F2010093F3011093F401E4C381EE91E03D
:102B00000E943F13DFC30F2EF0E06F2EF0E07F2E08
:102B1000FAE78F2EF4E49F2EF02D60925B01709205
:102B20005C0180925D0190925E0160914B01709119
:102B30004C0180914D0190914E0120E030E040EA3F
:102B400050E40E94261F69837A838B839C830F2E17
:102B5000F0E0EF2EF0E8FF2EFBE30F2FF5E41F2F40
:102B6000F02DED82FE820F831887CE010196BE0103
:102B70006B5F7F4F0E94741360914B0170914C0109
:102B800080914D0190914E0120E030E04AE753E4FE
:102B90000E94261F69877A878B879C87ED86FE8631
:102BA0000F87188BCE010996BE01635F7F4F0E948D
:102BB000741320E030E040E050E020934B0130936C
:102BC0004C0140934D0150934E0160925B01709215
:102BD0005C0180925D0190925E0180E090E0A0E84F
:102BE000BFE3898B9A8BAB8BBC8B6D8A7E8A8F8A75
:102BF000988ECE014196BE016B5E7F4F0E9474138A
:102C000060914B0170914C0180914D0190914E016A
:102C100020E030E040E251E40E94261F698F7A8F65
:102C20008B8F9C8F6D8E7E8E8F8E98A2CE01499653
:102C3000BE01635E7F4F0E94741320E030E040E0ED
:102C400050E020934B0130934C0140934D01509341
:102C50004E0160914F01709150018091510190910E
:102C6000520120E030E040EA50E40E94261F69A3B0
:102C70007AA38BA39CA3EDA2FEA20FA318A7CE015B
:102C80008196BE016B5D7F4F0E94A11360914F0141
:102C900070915001809151019091520120E030E0FB
:102CA0004AE753E40E94261F69A77AA78BA79CA72F
:102CB000EDA6FEA60FA718ABCE018996BE01635DF7
:102CC0007F4F0E94A11380E090E0A0E0B0E08093ED
:102CD0004F0190935001A0935101B0935201609223
:102CE0005B0170925C0180925D0190925E0120E038
:102CF00030E040E85FE329AB3AAB4BAB5CAB6DAA8D
:102D00007EAA8FAA98AECE01C196BE016B5C7F4FA2
:102D10000E94A11360914F01709150018091510167
:102D20009091520120E030E040E251E40E94261FE1
:102D300069AF7AAF8BAF9CAFFE01FD966082718266
:102D400082829382CE01C996BF010E94A11380E0C6
:102D500090E0A0E0B0E080934F0190935001A093E9
:102D60005101B09352010F2EF0E0AF2EF0E0BF2ED4
:102D7000F0EACF2EF1E4DF2EF02DA0925B01B092AD
:102D80005C01C0925D01D0925E0151E4452E512C50
:102D90004C0E5D1E6091530170915401809155015C
:102DA0009091560120E030E040E05FE30E94261F52
:102DB000D2016D937D938D939C931397FE01EB5BF2
:102DC000FF4F0F2EF0E0EF2EF0E0FF2EF8E40F2F74
:102DD000F2E41F2FF02DE082F18202831383C201FF
:102DE000BF010E94CE1349E4442E512C4C0E5D1EAF
:102DF0006091530170915401809155019091560159
:102E000020E030E04AE753E40E94261FF20160838D
:102E1000718382839383FE01E35BFF4FE082F18243
:102E200002831383C201BF010E94CE1320E030E071
:102E300040E050E0209353013093540140935501FA
:102E400050935601A0925B01B0925C01C0925D016B
:102E5000D0925E01DE01AF5ABF4F20E030E040E883
:102E60005FE32D933D934D935C931397FE01EB5AD3
:102E7000FF4FA082B182C282D382CD01BF010E94E6
:102E8000CE138E01075A1F4F609153017091540168
:102E9000809155019091560120E030E040E050E4EF
:102EA0000E94261FD8016D937D938D939C93139759
:102EB000FE01E35AFF4FA082B182C282D382C801D1
:102EC000BF010E94CE1320E030E040E050E02093AC
:102ED0005301309354014093550150935601609231
:102EE0005B0170925C0180925D0190925E01EAC18B
:102EF00090914A0180914901981709F0CEC1E09163
:102F00004A01F0E0EE0FFF1FEF5BFE4F0190F081F2
:102F1000E02DE855FF4F8081882309F0BEC18091E4
:102F20000B0290910C028531910509F467C086313E
:102F300091053CF48430910589F0449709F0A8C0CC
:102F400024C08B35910509F496C08C35910509F4A0
:102F500095C08A35910509F09BC089C06091110226
:102F600070911202809113029091140220E030E0DF
:102F700040E05FE30E94271F0E94F71F882777FD2C
:102F80008095982F0E94E31B93C0A1E4B1E028EF45
:102F900031E24BE453E40F2EF0E0AF2EF0E0BF2E11
:102FA000FEEFCF2EF5E4DF2EF02D0F2EFEE8EF2EF4
:102FB000F5E7FF2EFFE80F2FF1E41F2FF02D60E063
:102FC00070E080E89FE3ED91FD912083318342839F
:102FD00053832483358346835783A086B186C28674
:102FE000D386E486F58606871787608B718B828B84
:102FF000938BE1E0A934BE0731F75AC0A1E4B1E0F8
:103000002BE43AEE4FEF50E40F2EF0E0AF2EF0E05D
:10301000BF2EF0EACF2EF3E4DF2EF02D0F2EFAE6CE
:10302000EF2EFCEBFF2EF4E30F2FFFE31F2FF02D0D
:1030300060E070E080E89FE3ED91FD9120833183B3
:10304000428353832483358346835783A086B18686
:10305000C286D386E486F58606871787608B718BD8
:10306000828B938BF1E0A934BF0731F721C081E057
:10307000809325011DC0109225011AC0ABE4B1E078
:10308000E1EEF1E084E101900D928150E1F710C092
:1030900080EA95E064E071E00E94881C60910B0278
:1030A00070910C0280EA95E04AE050E00E94821D97
:1030B0008091090281FFCBC090914A018091490122
:1030C000981709F0F1C0E0914A01F0E0EE0FFF1F00
:1030D000EF5BFE4F0190F081E02DE855FF4F8081BE
:1030E000882309F0E1C080910D0290910E028C3688
:1030F00091057CF48A3691050CF0A9C088369105BB
:1031000089F0893691050CF040C0892B09F49FC0E5
:103110008EC08E37910509F44BC08F37910509F0A9
:1031200086C064C08091090290910A0292FF8FC00C
:10313000E0913601F0E0EE0FFF1FEE5CFE4F0081E4
:10314000118160913102709132028091330290912D
:1031500034020E94F71F9B01D80112967C936E9354
:1031600011978BE090E0FC012E9FC0012F9F900DE6
:103170003E9F900D11246AE070E00E94C521D801A5
:1031800014967C936E93139762C080EA95E06BE08F
:1031900071E00E94881CE0913601F0E0EE0FFF1F05
:1031A000EE5CFE4F808191810E949B07BC0149C06B
:1031B000E0913601F0E0EE0FFF1FEE5CFE4F008164
:1031C000118160911102709112028091130290910D
:1031D000140220E030E040E05FE30E94271F0E94DD
:1031E000F71F9B01AC01C80161E01DC0E0913601F1
:1031F000F0E0EE0FFF1FEE5CFE4F00811181609149
:10320000110270911202809113029091140220E039
:1032100030E040E05FE30E94271F0E94F71F9B0100
:10322000AC01C80160E0A9010E941C0810C080EA3E
:1032300095E06EE071E00E94881C60910D02709133
:103240000E0280EA95E04AE050E00E94821D8091E3
:10325000090290910A0296FF35C090914A0180912F
:103260004901981741F5E0914A01F0E0EE0FFF1F88
:10327000EF5BFE4F0190F081E02DE855FF4F80811C
:103280008823C9F490910F02911191E08091360149
:103290009817C1F09093360115C061E070E080E0AE
:1032A00090E00E94E31B24CE61E070E080E090E0BB
:1032B0000E94E31B01CF61E070E080E090E00E949B
:1032C000E31BCBCFC05ADF4F0FB6F894DEBF0FBE63
:1032D000CDBFCF91DF911F910F91FF90EF90DF90C5
:1032E000CF90BF90AF909F908F907F906F905F90A6
:1032F0004F90089580EA95E00E949D1E882311F169
:1033000080EA95E00E94B11E809322018D3019F46D
:103310008AE0809322019091220190329CF09B33AD
:1033200019F481E08093E0018091E001882351F459
:103330008091DF01E82FF0E0E15AFE4F90838F5F2C
:103340008093DF018091DF0187FF04C01092DF01CD
:103350001092E0016091DF01662351F1809122011A
:103360008A3031F570E0FB01E15AFE4F10828FE5A3
:1033700091E00E94FB131092DF011092E001809116
:103380003701882379F080EA95E065E171E00E94D9
:10339000881C80EA95E067E371E00E94771D109237
:1033A0003701089580EA95E069E171E00E94771D98
:1033B00008950E94DB070E947A190895EF92FF9208
:1033C0000F931F936FE6E62EF12CF70180818D7F1E
:1033D00080830E94D9041092370186E592E0909391
:1033E0003301809332018DE392E090933501809315
:1033F0003401109236011092490110924A018FE671
:1034000092E0909342018093410188E193E0909390
:1034100044018093430181EC93E0909346018093B3
:1034200045018AE694E09093480180934701109209
:10343000DF011092E00180E090E0A0E0B0E0809336
:103440004B0190934C01A0934D01B0934E0180939A
:103450004F0190935001A0935101B093520180937A
:10346000530190935401A0935501B093560180935A
:10347000570190935801A0935901B0935A0180E0ED
:1034800090E0AAE7B4E480935B0190935C01A09381
:103490005D01B0935E0100EA15E0C80140E05BE425
:1034A00060E070E00E94A41DC8016CE171E00E9420
:1034B000771D68EE73E080E090E00E945705F70109
:1034C0008081826080831F910F91FF90EF9008951B
:1034D000282F30E0C90182559F4FFC019491265658
:1034E0003F4FF9018491882391F0E82FF0E0EE0F2F
:1034F000FF1FE458FF4FA591B491662329F48C91E6
:10350000909589238C9308958C91892B8C930895A1
:10351000482F50E0CA018E539F4FFC012491CA01ED
:1035200082559F4FFC01949146565F4FFA013491AA
:103530003323D1F1222331F1233021F48091800013
:103540008F7705C0243031F4809180008F7D809387
:10355000800018C0213019F484B58F7704C0223060
:1035600021F484B58F7D84BD0DC0263021F4809177
:10357000B0008F7705C0273029F48091B0008F7D8F
:103580008093B000E32FF0E0EE0FFF1FEA57FF4FEC
:10359000A591B491662329F48C91909589238C93FD
:1035A00008958C91892B8C930895682F70E0CB013E
:1035B0008E539F4FFC012491CB0182559F4FFC01FC
:1035C000449166567F4FFB019491992319F420E0B2
:1035D00030E038C0222331F1233021F48091800083
:1035E0008F7705C0243031F4809180008F7D8093E7
:1035F000800018C0213019F484B58F7704C02230C0
:1036000021F484B58F7D84BD0DC0263021F48091D6
:10361000B0008F7705C0273029F48091B0008F7DEE
:103620008093B000892F90E0880F991F80579F4F9B
:10363000FC01A591B4918C9120E030E0842311F03D
:1036400021E030E0C901089587709091260192959C
:10365000990F990F907C982B90937C0080917A0021
:10366000806480937A0080917A0086FDFCCF20915F
:10367000780040917900942F80E030E0282B392B9E
:10368000C90108951F93CF93DF93182FEB0161E0D9
:103690000E94681AE12FF0E0EE53FF4F84918330CF
:1036A00051F480918000806880938000D0938900DD
:1036B000C09388003CC0843051F4809180008062C7
:1036C00080938000D0938B00C0938A0030C08130FB
:1036D00039F4209729F184B5806884BDC7BD27C01F
:1036E000823039F42097E1F084B5806284BDC8BD92
:1036F0001EC0863041F48091B00080688093B00095
:10370000C093B30014C0873041F48091B000806250
:103710008093B000C093B4000AC0C038D1051CF437
:10372000812F60E002C0812F61E00E94881ADF9142
:10373000CF911F9108951F920F920FB60F921124EF
:103740002F933F938F939F93AF93BF9380911705D0
:1037500090911805A0911905B0911A0530911B059B
:103760000196A11DB11D232F2D5F2D3720F02D5760
:103770000196A11DB11D20931B0580931705909301
:103780001805A0931905B0931A058091130590911F
:103790001405A0911505B09116050196A11DB11D46
:1037A0008093130590931405A0931505B093160507
:1037B000BF91AF919F918F913F912F910F900FBE2D
:1037C0000F901F901895EF92FF920F931F937B011C
:1037D0008C018FB7F89440911705509118056091AE
:1037E000190570911A058FBF2FB7F89480911705AE
:1037F00090911805A0911905B0911A052FBF841B4F
:10380000950BA60BB70BE816F9060A071B0760F71E
:103810001F910F91FF90EF900895019739F0880F55
:10382000991F880F991F02970197F1F708957894CF
:1038300084B5826084BD84B5816084BD85B58260B5
:1038400085BD85B5816085BDEEE6F0E08081816053
:103850008083E1E8F0E08081826080838081816004
:103860008083E0E8F0E0808181608083E1EBF0E03C
:10387000808184608083E0EBF0E0808181608083E0
:10388000EAE7F0E0808184608083808182608083C9
:103890008081816080838081806880831092C100F4
:1038A00008950F931F93CF93DF938C01EB0109C011
:1038B0002196D801ED91FC910190F081E02DC80195
:1038C000099568816623A1F7DF91CF911F910F9130
:1038D0000895EF92FF920F931F93CF93DF938C0184
:1038E0007B01EA010CC0D7016D917D01D801ED91FA
:1038F000FC910190F081E02DC80109952197209756
:1039000091F7DF91CF911F910F91FF90EF90089564
:10391000DC01ED91FC910280F381E02D0995089581
:103920002F923F924F925F926F927F928F929F92CF
:10393000AF92BF92CF92DF92EF92FF920F931F93BD
:10394000DF93CF93CDB7DEB7A0970FB6F894DEBF65
:103950000FBECDBF1C016A017B01411551056105F8
:10396000710549F440E350E060E070E020E030E0B1
:103970000E942A1D56C0882499245401422E5524A1
:103980006624772401E010E00C0F1D1F080D191D9F
:10399000C701B601A30192010E94D821F8016083FA
:1039A0000894811C911CA11CB11CC701B601A30184
:1039B00092010E94D821C901DA016C017D01C11474
:1039C000D104E104F104F1F681E0E82EF12CEC0ED3
:1039D000FD1EE80CF91C3E010894611C711CD50108
:1039E000C4010197A109B1096C01C818D90816C012
:1039F000F601EE0DFF1D40814A3010F4405D01C01C
:103A0000495C552747FD5095652F752FC10120E072
:103A100030E00E942A1D0894E108F1086E147F042A
:103A200039F7A0960FB6F894DEBF0FBECDBFCF9189
:103A3000DF911F910F91FF90EF90DF90CF90BF909B
:103A4000AF909F908F907F906F905F904F903F903E
:103A50002F900895EF92FF920F931F93CF93DF93D0
:103A6000EC017A018B012115310541F4E881F981DE
:103A70000190F081E02D642F09951BC02A3031059B
:103A8000B1F477FF10C04DE250E060E070E020E05C
:103A900030E00E942A1D10950095F094E094E11CFE
:103AA000F11C011D111DCE01B801A7012AE00E94E1
:103AB000901CDF91CF911F910F91FF90EF9008958F
:103AC0000F931F938C014DE050E060E070E020E028
:103AD00030E00E942A1DC8014AE050E060E070E03A
:103AE00020E030E00E942A1D1F910F9108950F934E
:103AF0001F938C010E94881CC8010E94601D1F91A9
:103B00000F910895CF92DF92EF92FF920F931F9340
:103B10008C016B019A01EE24D7FCE094FE2CB701D6
:103B2000A6010E942A1DC8010E94601D1F910F91CD
:103B3000FF90EF90DF90CF9008950E94171C0E9495
:103B4000DE190E94D919FDCF5F926F927F928F92FA
:103B50009F92AF92BF92CF92DF92EF92FF920F931C
:103B60001F93CF93DF93EC013A014B01413482E480
:103B700058078FE0680780E078070CF07FC060E8A6
:103B800074E88EE190E0A40193010E94FA21215093
:103B9000304040405040CA01B90122E030E040E0EE
:103BA00050E00E94FA2159016A01A6019501209571
:103BB00030954095509594E0220F331F441F551FB8
:103BC0009A95D1F760E074E284EF90E00E94FA21C8
:103BD000CA01B9012FEF30E040E050E00E94A62179
:103BE000A40193010E94FA21C90181509F4F181628
:103BF00019061CF4522E5A9403C055245394521A99
:103C000060E079E08DE390E0A40193010E94FA2145
:103C10002150304040405040CA01B90122E030E01C
:103C200040E050E00E94FA21209530954095509553
:103C300083E0220F331F441F551F8A95D1F760E0A0
:103C400074E284EF90E00E94FA21CA01B9012FEFDB
:103C500030E040E050E00E94A621A40193010E94C0
:103C6000FA21C90181509F4F181619061CF4822FA2
:103C7000815002C081E0821B851500F5E885F98539
:103C800081E090E00A8802C0880F991F0A94E2F749
:103C9000808360E079E08DE390E0A40193010E94CD
:103CA000FA212150304040405040CA01B90122E081
:103CB00030E040E050E00E94FA2104C0E885F98538
:103CC00010829501EC81FD813083EE81FF8120839C
:103CD000EA85FB85208141E050E0CA010E8402C0E4
:103CE000880F991F0A94E2F7282B2083EA85FB8529
:103CF0002081CA010F8402C0880F991F0A94E2F73D
:103D0000282B2083EA85FB858081088802C0440F28
:103D1000551F0A94E2F7842B8083DF91CF911F9186
:103D20000F91FF90EF90DF90CF90BF90AF909F905A
:103D30008F907F906F905F900895DC011296ED91C7
:103D4000FC911397E058FF4F8191919180589F4FBC
:103D500020813181821B930B60E870E00E94C521B5
:103D60000895CF93DF93DC011296ED91FC911397A8
:103D7000EF01CE57DF4F48815981E058FF4F8081D6
:103D80009181E058F0408417950719F42FEF3FEF29
:103D90000CC0E40FF51F2081CA01019660E870E0B5
:103DA0000E94C5219983888330E0C901DF91CF91BA
:103DB0000895FC01A085B18521898C9190E0022EA7
:103DC00002C0959587950A94E2F780FFF6CF0484A8
:103DD000F585E02D608308958BE291E09093A10535
:103DE0008093A0058CE195E09093A3058093A205B4
:103DF00085EC90E09093A5058093A40584EC90E079
:103E00009093A7058093A60580EC90E09093A90578
:103E10008093A80581EC90E09093AB058093AA0570
:103E200086EC90E09093AD058093AC0584E08093A0
:103E3000AE0583E08093AF0587E08093B00585E011
:103E40008093B10581E08093B20508955058BB2757
:103E5000AA270ED075C166D130F06BD120F031F4B5
:103E60009F3F11F41EF45BC10EF4E095E7FB51C1D6
:103E7000E92F77D180F3BA17620773078407950794
:103E800018F071F49EF58FC10EF4E0950B2EBA2F49
:103E9000A02D0B01B90190010C01CA01A001112450
:103EA000FF27591B99F0593F50F4503E68F11A16FC
:103EB000F040A22F232F342F4427585FF3CF46958D
:103EC00037952795A795F0405395C9F77EF41F16AF
:103ED000BA0B620B730B840BBAF09150A1F0FF0F79
:103EE000BB1F661F771F881FC2F70EC0BA0F621F65
:103EF000731F841F48F4879577956795B795F79555
:103F00009E3F08F0B3CF9395880F08F09927EE0FE6
:103F1000979587950895D9D008F481E008950CD03D
:103F20000FC107D140F0FED030F021F45F3F19F00F
:103F3000F0C0511139C1F3C014D198F39923C9F3DA
:103F40005523B1F3951B550BBB27AA27621773079F
:103F5000840738F09F5F5F4F220F331F441FAA1F53
:103F6000A9F333D00E2E3AF0E0E830D09150504013
:103F7000E695001CCAF729D0FE2F27D0660F771FC1
:103F8000881FBB1F261737074807AB07B0E809F0A3
:103F9000BB0B802DBF01FF2793585F4F2AF09E3F38
:103FA000510568F0B6C000C15F3FECF3983EDCF30A
:103FB000869577956795B795F7959F5FC9F7880FB1
:103FC000911D9695879597F90895E1E0660F771F03
:103FD000881FBB1F621773078407BA0720F0621B94
:103FE000730B840BBA0BEE1F88F7E095089504D08D
:103FF0006894B111D9C00895BCD088F09F5790F053
:10400000B92F9927B751A0F0D1F0660F771F881FFD
:10401000991F1AF0BA95C9F712C0B13081F0C3D018
:10402000B1E00895C0C0672F782F8827B85F39F0B6
:10403000B93FCCF3869577956795B395D9F73EF45C
:1040400090958095709561957F4F8F4F9F4F089504
:10405000E89409C097FB3EF4909580957095619522
:104060007F4F8F4F9F4F9923A9F0F92F96E9BB27D8
:104070009395F695879577956795B795F111F8CF54
:10408000FAF4BB0F11F460FF1BC06F5F7F4F8F4FBF
:104090009F4F16C0882311F096E911C0772321F0B5
:1040A0009EE8872F762F05C0662371F096E8862F4D
:1040B00070E060E02AF09A95660F771F881FDAF7A4
:1040C000880F9695879597F90895990F0008550FD1
:1040D000AA0BE0E8FEEF16161706E807F907C0F08E
:1040E00012161306E407F50798F0621B730B840B96
:1040F000950B39F40A2661F0232B242B252B21F470
:1041000008950A2609F4A140A6958FEF811D811D0F
:10411000089597F99F6780E870E060E008959FEF49
:1041200080EC089500240A9416161706180609064E
:10413000089500240A94121613061406050608951D
:10414000092E0394000C11F4882352F0BB0F40F4A5
:10415000BF2B11F460FF04C06F5F7F4F8F4F9F4FE5
:10416000089557FD9058440F551F59F05F3F71F067
:104170004795880F97FB991F61F09F3F79F08795CE
:104180000895121613061406551FF2CF4695F1DF57
:1041900008C0161617061806991FF1CF86957105E7
:1041A000610508940895E894BB2766277727CB011B
:1041B00097F908958ADF08F48FEF08950BD0C0CFE8
:1041C000B1DF28F0B6DF18F0952309F0A2CFA7CF12
:1041D0001124EACFC6DFA0F3959FD1F3950F50E0ED
:1041E000551F629FF001729FBB27F00DB11D639FA9
:1041F000AA27F00DB11DAA1F649F6627B00DA11D4F
:10420000661F829F2227B00DA11D621F739FB00DF4
:10421000A11D621F839FA00D611D221F749F332764
:10422000A00D611D231F849F600D211D822F762FFD
:104230006A2F11249F5750408AF0E1F088234AF0FA
:10424000EE0FFF1FBB1F661F771F881F9150504046
:10425000A9F79E3F510570F05CCFA6CF5F3FECF30E
:10426000983EDCF3869577956795B795F795E79532
:104270009F5FC1F7FE2B880F911D9695879597F943
:10428000089511F40EF44BCF4AC073DFD0F3992395
:10429000D9F3CEF39F57550B87FF51D0569597957D
:1042A000B0E020F4660F771F881FBB1F1F930F938A
:1042B00000249001A0018001F001A0E80E0F1F1F53
:1042C0000A1E511D601B710B8009B50B48F4600F6D
:1042D000711F801DB51F0E1B1F0B0A0A510907C055
:1042E0002E0F3F1F4A1F0E0F1F1F0A1E511D660F64
:1042F000771F881FBB1FA695F795E795F8F6061759
:10430000170708065B07211D311D411D0F911F91E5
:10431000B901842F9158880F9695879508959F3FEE
:1043200049F0915028F4869577956795B7959F5FEA
:1043300080389F4F880F9695879597F908959150EB
:104340005040660F771F881FD2F70895629FD001F3
:10435000739FF001829FE00DF11D649FE00DF11D40
:10436000929FF00D839FF00D749FF00D659FF00DEF
:104370009927729FB00DE11DF91F639FB00DE11DDC
:10438000F91FBD01CF011124089597FB092E0726BF
:104390000AD077FD04D049D006D000201AF47095D9
:1043A00061957F4F0895F6F7909581959F4F0895F9
:1043B000A1E21A2EAA1BBB1BFD010DC0AA1FBB1F29
:1043C000EE1FFF1FA217B307E407F50720F0A21B9B
:1043D000B30BE40BF50B661F771F881F991F1A9408
:1043E00069F760957095809590959B01AC01BD0132
:1043F000CF01089597FB092E05260ED057FD04D056
:10440000D7DF0AD0001C38F450954095309521959F
:104410003F4F4F4F5F4F0895F6F7909580957095F9
:1044200061957F4F8F4F9F4F0895AA1BBB1B51E192
:1044300007C0AA1FBB1FA617B70710F0A61BB70B14
:10444000881F991F5A95A9F780959095BC01CD01B9
:104450000895EE0FFF1F0590F491E02D099491113E
:1044600006C0803219F089508550D0F708959927F9
:10447000882708952F923F924F925F926F927F927A
:104480008F929F92AF92BF92CF92DF92EF92FF9264
:104490000F931F93CF93DF93CDB7DEB7CA1BDB0B10
:1044A0000FB6F894DEBF0FBECDBF09942A883988B5
:1044B00048885F846E847D848C849B84AA84B984BC
:1044C000C884DF80EE80FD800C811B81AA81B981C8
:1044D000CE0FD11D0FB6F894DEBF0FBECDBFED01DC
:0644E0000895F894FFCFDF
:1044E600453A20006875683F204700543A004875F1
:1044F600683F204D006F6B20006F6B007374617214
:1045060074003FFFFF010100000000D91E511C6925
:024516001C0087
:00000001FF
